:100000000C9438000C9453000C9453000C9453003F
:100010000C9453000C9453000C9453000C94530014
:100020000C9453000C9453000C9453000C94530004
:100030000C9453000C9453000C9453000C945300F4
:100040000C9453000C94C3020C9453000C94530072
:100050000C94E40F0C9453000C9453000C94530034
:100060000C9453000C9453000C9453000C945300C4
:1000700011241FBECFEFD4E0DEBFCDBF13E0A0E060
:10008000B1E0ECEBF4E202C005900D92A43AB107A6
:10009000D9F714E0A4EAB3E001C01D92A139B10779
:1000A000E1F70C9472000C940000CF93DF93CDB76E
:1000B000DEB7E4E3F0E08FEF8083EAE3F0E08EE286
:1000C0008083ABE3B0E0EBE3F0E0808182608C936F
:1000D000ABE3B0E0EBE3F0E0808180628C93DF91F2
:1000E000CF910895CF93DF93CDB7DEB70E9455002F
:1000F0000E94B4020E94E20E7894A5E3B0E0E5E32A
:10010000F0E0808181608C930E9487020E94FF0250
:100110000E9449030E9493030E94DD030E9427046A
:100120000E9471040E94BB040E9405050E944F05B5
:100130000E9499050E94E3050E94580700C0809123
:10014000A603813031F41092A6030E94C4110E94CC
:10015000D3118091B3038130E1F4A5E3B0E0E5E38E
:10016000F0E0808184608C930E94EE0D0E947610F6
:100170000E94F8070E940D090E94410A0E94A406ED
:100180000E948907A5E3B0E0E5E3F0E080818B7F82
:100190008C938091A403813091F61092A4030E9465
:1001A0002D06CDCFCF93DF93CDB7DEB764E084E0EB
:1001B0000E94EF006CE480E00E94EF001092A60322
:1001C0008091A6038823E1F36AE08CE60E94EF00A9
:1001D00060E085E00E94EF00DF91CF910895CF931A
:1001E000DF93CDB7DEB724970FB6F894DEBF0FBE0E
:1001F000CDBF8B836C83ABE3B0E0EBE3F0E08081B9
:100200008D7F8C9387E08A8340C0ABE3B0E0EBE363
:10021000F0E08081877F8C930000000000000000E8
:100220008A81282F332727FD309581E090E0022E28
:1002300002C0880F991F0A94E2F7982F8B818923B7
:1002400089838981882341F0ABE3B0E0EBE3F0E000
:10025000808184608C9307C0ABE3B0E0EBE3F0E017
:1002600080818B7F8C930000000000000000ABE3D6
:10027000B0E0EBE3F0E0808188608C930000000048
:10028000000000008A8181508A838A8188230CF0D3
:10029000BCCF87E08A8340C0ABE3B0E0EBE3F0E0A3
:1002A0008081877F8C9300000000000000008A811D
:1002B000282F332727FD309581E090E0022E02C0E1
:1002C000880F991F0A94E2F7982F8C8189238983DC
:1002D0008981882341F0ABE3B0E0EBE3F0E080817B
:1002E00084608C9307C0ABE3B0E0EBE3F0E0808187
:1002F0008B7F8C930000000000000000ABE3B0E0B7
:10030000EBE3F0E0808188608C9300000000000047
:1003100000008A8181508A838A8188230CF0BCCFB7
:10032000ABE3B0E0EBE3F0E08081877F8C93ABE35D
:10033000B0E0EBE3F0E080818B7F8C93ABE3B0E047
:10034000EBE3F0E0808182608C9324960FB6F89402
:10035000DEBF0FBECDBFDF91CF910895CF93DF9366
:10036000CDB7DEB724970FB6F894DEBF0FBECDBF72
:100370008C83ABE3B0E0EBE3F0E080818D7F8C9386
:1003800087E08A834CC0ABE3B0E0EBE3F0E0808130
:10039000877F8C9300000000000000000000000038
:1003A000000000008A81282F332727FD309581E047
:1003B00090E0022E02C0880F991F0A94E2F7982F4E
:1003C0008C8189238B838B81181644F4ABE3B0E0D6
:1003D000EBE3F0E0808184608C9307C0ABE3B0E096
:1003E000EBE3F0E080818B7F8C9300000000000045
:1003F00000000000000000000000ABE3B0E0EBE311
:10040000F0E0808188608C93000000000000000014
:1004100000000000000000008A8181508A838A81E8
:1004200088230CF0B0CF1B82ABE3B0E0EBE3F0E04D
:100430008081877F8C930000000000000000000096
:1004400000000000000087E08A833DC0ABE3B0E01D
:10045000EBE3F0E0808188608C93E9E3F0E0808159
:1004600089838981992780719070181619068CF4F8
:100470008A81282F332727FD309581E090E0022ED6
:1004800002C0880F991F0A94E2F7982F8B81892B5D
:100490008B8300000000000000000000000000004E
:1004A0000000ABE3B0E0EBE3F0E08081877F8C936A
:1004B000000000000000000000000000000000003C
:1004C0008A8181508A838A8188230CF0BFCFABE375
:1004D000B0E0EBE3F0E08081877F8C93ABE3B0E0AA
:1004E000EBE3F0E080818B7F8C93ABE3B0E0EBE358
:1004F000F0E0808182608C938B81992724960FB6DF
:10050000F894DEBF0FBECDBFDF91CF910895CF939A
:10051000DF93CDB7DEB70E94D2001092A403809182
:10052000A4038823E1F30E946A060E94130C109230
:10053000A4038091A4038823E1F31092A403809183
:10054000A4038823E1F31092A40364E084E00E94F2
:10055000EF006CE480E00E94EF000E942D060E94F4
:10056000C306DF91CF910895CF93DF93CDB7DEB768
:10057000E3E5F0E082E08083E9E5F0E082E080837B
:10058000DF91CF9108951F920F920FB60F92112411
:100590008F93CF93DF93CDB7DEB78091A8038F5FA2
:1005A0008093A8038091A803883409F581E08093A3
:1005B000A7031092A80380914C048F5F80934C0492
:1005C00080914C04843629F410924C0481E080938D
:1005D000A40380914B048F5F80934B0480914B0464
:1005E0008A3029F410924B0481E08093A603DF91B6
:1005F000CF918F910F900FBE0F901F901895CF93B2
:10060000DF93CDB7DEB762E480E00E94EF00109286
:10061000A4038091A4038823E1F31092A4036EEA5B
:1006200089E00E94EF001092A6038091A603882320
:10063000E1F31092A60310924D0416C080914D0470
:10064000682F8AE00E94EF0080914D049927FC01F9
:10065000E95CFE4F8081682F8BE00E94EF00809163
:100660004D048F5F80934D0480914D04863330F3A9
:1006700060EA88E00E94EF001092A6038091A60332
:100680008823E1F36CE480E00E94EF00DF91CF91DA
:100690000895CF93DF93CDB7DEB762E480E00E9488
:1006A000EF001092A4038091A4038823E1F3109239
:1006B000A4036FEA89E00E94EF001092A6038091E4
:1006C000A6038823E1F31092A60310924D0416C0EE
:1006D00080914D04682F8AE00E94EF0080914D04C4
:1006E0009927FC01E159FE4F8081682F8BE00E9421
:1006F000EF0080914D048F5F80934D0480914D04F5
:10070000863330F360EA88E00E94EF001092A6037F
:100710008091A6038823E1F36CE480E00E94EF005F
:10072000DF91CF910895CF93DF93CDB7DEB762E429
:1007300080E00E94EF001092A4038091A40388231C
:10074000E1F31092A40360EB89E00E94EF001092A5
:10075000A6038091A6038823E1F31092A6031092CA
:100760004D0416C080914D04682F8AE00E94EF006E
:1007700080914D049927FC01E955FE4F8081682F37
:100780008BE00E94EF0080914D048F5F80934D04B9
:1007900080914D04863330F360EA88E00E94EF00D8
:1007A0001092A6038091A6038823E1F36CE480E015
:1007B0000E94EF00DF91CF910895CF93DF93CDB7E3
:1007C000DEB762E480E00E94EF001092A403809103
:1007D000A4038823E1F31092A40361EB89E00E9453
:1007E000EF001092A6038091A6038823E1F31092F4
:1007F000A60310924D0416C080914D04682F8AE024
:100800000E94EF0080914D049927FC01E152FE4FB8
:100810008081682F8BE00E94EF0080914D048F5FF4
:1008200080934D0480914D04863330F360EA88E074
:100830000E94EF001092A6038091A6038823E1F3A3
:100840006CE480E00E94EF00DF91CF910895CF9398
:10085000DF93CDB7DEB762E480E00E94EF00109234
:10086000A4038091A4038823E1F31092A40362EB14
:1008700089E00E94EF001092A6038091A6038823CE
:10088000E1F31092A60310924D0416C080914D041E
:10089000682F8AE00E94EF0080914D049927FC01A7
:1008A000E95EFD4F8081682F8BE00E94EF00809110
:1008B0004D048F5F80934D0480914D04863330F357
:1008C00060EA88E00E94EF001092A6038091A603E0
:1008D0008823E1F36CE480E00E94EF00DF91CF9188
:1008E0000895CF93DF93CDB7DEB762E480E00E9436
:1008F000EF001092A4038091A4038823E1F31092E7
:10090000A40363EB89E00E94EF001092A60380919C
:10091000A6038823E1F31092A60310924D0416C09B
:1009200080914D04682F8AE00E94EF0080914D0471
:100930009927FC01E15BFD4F8081682F8BE00E94CD
:10094000EF0080914D048F5F80934D0480914D04A2
:10095000863330F360EA88E00E94EF001092A6032D
:100960008091A6038823E1F36CE480E00E94EF000D
:10097000DF91CF910895CF93DF93CDB7DEB762E4D7
:1009800080E00E94EF001092A4038091A4038823CA
:10099000E1F31092A40364EB89E00E94EF0010924F
:1009A000A6038091A6038823E1F31092A603109278
:1009B0004D0416C080914D04682F8AE00E94EF001C
:1009C00080914D049927FC01E957FD4F8081682FE4
:1009D0008BE00E94EF0080914D048F5F80934D0467
:1009E00080914D04863330F360EA88E00E94EF0086
:1009F0001092A6038091A6038823E1F36CE480E0C3
:100A00000E94EF00DF91CF910895CF93DF93CDB790
:100A1000DEB762E480E00E94EF001092A4038091B0
:100A2000A4038823E1F31092A40365EB89E00E94FC
:100A3000EF001092A6038091A6038823E1F31092A1
:100A4000A60310924D0416C080914D04682F8AE0D1
:100A50000E94EF0080914D049927FC01E154FD4F65
:100A60008081682F8BE00E94EF0080914D048F5FA2
:100A700080934D0480914D04863330F360EA88E022
:100A80000E94EF001092A6038091A6038823E1F351
:100A90006CE480E00E94EF00DF91CF910895CF9346
:100AA000DF93CDB7DEB762E480E00E94EF001092E2
:100AB000A4038091A4038823E1F31092A40366EBBE
:100AC00089E00E94EF001092A6038091A60388237C
:100AD000E1F31092A60310924D0416C080914D04CC
:100AE000682F8AE00E94EF0080914D049927FC0155
:100AF000E950FD4F8081682F8BE00E94EF008091CC
:100B00004D048F5F80934D0480914D04863330F304
:100B100060EA88E00E94EF001092A6038091A6038D
:100B20008823E1F36CE480E00E94EF00DF91CF9135
:100B30000895CF93DF93CDB7DEB762E480E00E94E3
:100B4000EF001092A4038091A4038823E1F3109294
:100B5000A40367EB89E00E94EF001092A603809146
:100B6000A6038823E1F31092A60310924D0416C049
:100B700080914D04682F8AE00E94EF0080914D041F
:100B80009927FC01E15DFC4F8081682F8BE00E947A
:100B9000EF0080914D048F5F80934D0480914D0450
:100BA000863330F360EA88E00E94EF001092A603DB
:100BB0008091A6038823E1F36CE480E00E94EF00BB
:100BC000DF91CF910895CF93DF93CDB7DEB762E485
:100BD00080E00E94EF001092A4038091A403882378
:100BE000E1F31092A40368EB89E00E94EF001092F9
:100BF000A6038091A6038823E1F31092A603109226
:100C00004D0416C080914D04682F8AE00E94EF00C9
:100C100080914D049927FC01E959FC4F8081682F90
:100C20008BE00E94EF0080914D048F5F80934D0414
:100C300080914D04863330F360EA88E00E94EF0033
:100C40001092A6038091A6038823E1F36CE480E070
:100C50000E94EF00DF91CF910895CF93DF93CDB73E
:100C6000DEB789ED80934D0413C060E085E00E94FB
:100C7000EF0080914D04682F86E00E94EF0064E54C
:100C800087E00E94EF0080914D048F5F80934D04B8
:100C900080914D048C3D48F385EE80934D0413C044
:100CA00060E085E00E94EF0080914D04682F86E0AF
:100CB0000E94EF0064E587E00E94EF0080914D0400
:100CC0008F5F80934D0480914D04883E48F3DF91FF
:100CD000CF910895CF93DF93CDB7DEB764970FB66A
:100CE000F894DEBF0FBECDBF8DE589838EE58A8384
:100CF0008FE58B8389E48C838BE58D838DE18E83F7
:100D00008CE58F83188680E2898789E28A8786E36B
:100D10008B8781E48C878AE08D8781E48E8781E0F0
:100D20008F8786E2888B20E1CE010196AC0162E0DC
:100D300087E00E94EE0664960FB6F894DEBF0FBE01
:100D4000CDBFDF91CF910895CF93DF93CDB7DEB7BD
:100D500060E085E00E94EF006FEC86E00E94EF000B
:100D60006CE887E00E94EF0061E085E00E94EF0000
:100D70006BE086E00E94EF006DE887E00E94EF00E4
:100D8000DF91CF910895CF93DF93CDB7DEB760E0C9
:100D900085E00E94EF0060E286E00E94EF0060E8DC
:100DA00087E00E94EF0060E085E00E94EF006EE3C4
:100DB00086E00E94EF0064E887E00E94EF0060E0B8
:100DC00085E00E94EF006CE586E00E94EF0068E895
:100DD00087E00E94EF00DF91CF910895CF93DF93DA
:100DE000CDB7DEB72D970FB6F894DEBF0FBECDBFDF
:100DF00089876A875C874B872D878A85282F3327C9
:100E00008EE190E0A901489F9001499F300D589FC5
:100E1000300D112489859927820F931F98878F831E
:100E20008D85282F33278F819885820F931F9E836E
:100E30008D8310924D048F8198859C838B8328C06D
:100E40008B818A838B819C81892F992789836981F2
:100E500085E00E94EF006A8186E00E94EF004091E9
:100E60004D04842F99279C018B859C85F901E80FFF
:100E7000F91F8081982F842F8F5F80934D04692FF5
:100E800087E00E94EF008B819C8101969C838B837D
:100E90002B813C818D819E812817390788F22D9600
:100EA0000FB6F894DEBF0FBECDBFDF91CF9108958E
:100EB000CF93DF93CDB7DEB781E091E029E0AC01BD
:100EC0006EE083E00E94EE06DF91CF910895CF930C
:100ED000DF93CDB7DEB722970FB6F894DEBF0FBE13
:100EE000CDBF8A838A81882321F48A8186528983AF
:100EF00003C08A81805389838981992787FD9095D2
:100F000022960FB6F894DEBF0FBECDBFDF91CF9112
:100F100008950F931F93CF93DF93CDB7DEB72D972F
:100F20000FB6F894DEBF0FBECDBF80915A049091EA
:100F30005B042EE130E0B9010E943712CB019B83A4
:100F40008A83CE0104962A813B814AE050E0BC01AD
:100F5000C9010E940612CE010496DC01FD01019038
:100F60000020E9F73197CF018A1B9B0B89831092F0
:100F70004D041CC080914D04082F112780914D0411
:100F8000282F3327CE010496FC01E20FF31F808146
:100F90000E946707282FCE010996FC01E00FF11F80
:100FA000208380914D048F5F80934D0480914D0488
:100FB000282F33278981992787FD9095281739078E
:100FC000CCF2298199818BE0382F391BCE0109960B
:100FD000AC016EE0832F0E94EE062D960FB6F894BA
:100FE000DEBF0FBECDBFDF91CF911F910F9108954E
:100FF000CF93DF93CDB7DEB729970FB6F894DEBF56
:101000000FBECDBF80916204909163048E559040D5
:101010009C838B838B819C8123E030E0B9010E940B
:101020003712CB019A83898389819A818A3091050D
:1010300024F089E090E09A83898389819A819923B9
:1010400014F41A8219822091AC033091AD03898186
:101050009A818217930709F4D7C089819A818230D7
:1010600091052CF460E184E00E94EF0004C060E090
:1010700084E00E94EF0089819A819093AD03809370
:10108000AC0380E88D8384E88E8388E88F83898130
:101090009A8199878887888599858430910509F494
:1010A0005FC08885998585309105DCF488859985B0
:1010B0008130910509F43FC088859985823091057A
:1010C0002CF488859985009779F173C08885998576
:1010D00082309105B9F18885998583309105C9F1F0
:1010E00068C0888599858730910509F44EC0888548
:1010F0009985883091055CF48885998585309105BE
:10110000B1F18885998586309105C1F152C08885F5
:1011100099858830910509F43FC088859985893083
:10112000910509F440C045C080E88D8384E88E8332
:1011300088E88F833EC081E88D8384E88E8388E8C9
:101140008F8337C082E88D8384E88E8388E88F831D
:1011500030C083E88D8384E88E8388E88F8329C03C
:1011600083E88D8385E88E8388E88F8322C083E8B7
:101170008D8386E88E8388E88F831BC083E88D8308
:1011800087E88E8388E88F8314C083E88D8387E89F
:101190008E8389E88F830DC083E88D8387E88E83F3
:1011A0008AE88F8306C083E88D8387E88E838BE887
:1011B0008F8360E085E00E94EF0060E286E00E949D
:1011C000EF008D81682F87E00E94EF0060E085E0EE
:1011D0000E94EF006EE386E00E94EF008E81682F90
:1011E00087E00E94EF0060E085E00E94EF006CE580
:1011F00086E00E94EF008F81682F87E00E94EF0059
:1012000060E084E00E94EF0029960FB6F894DEBFFC
:101210000FBECDBFDF91CF910895CF93DF93CDB7B0
:10122000DEB726970FB6F894DEBF0FBECDBF809114
:1012300052049091530426E130E0B9010E94371224
:10124000CB0106969E838D838D819E8199230CF41C
:1012500046C08D819E812AE030E0B9010E9437129C
:10126000CB018A838D819E812AE030E0B9010E9402
:1012700037128983898186958C5F89838A81282F9B
:10128000332786E890E0821B930B9C838B8320910D
:101290000D0130910E018B819C818217930761F0C3
:1012A00080910D0190910E010E94C6098B819C8155
:1012B00069810E94000A0AC09091B1038981981740
:1012C00029F08B819C8169810E94000A8981809329
:1012D000B1038B819C8190930E0180930D018D81D0
:1012E0009E8199230CF049C08D819E8190958195B6
:1012F0009F4F9E838D838D819E812AE030E0B901CE
:101300000E943712CB018A838D819E812AE030E0D2
:10131000B9010E94371289838981869589838A81E0
:1013200099278A579F4F9C838B8320910D01309181
:101330000E018B819C818217930761F080910D01D2
:1013400090910E010E94C6098B819C8169810E9447
:10135000000A0AC09091B1038981981729F08B8106
:101360009C8169810E94000A89818093B1038B81ED
:101370009C8190930E0180930D0126960FB6F894F0
:10138000DEBF0FBECDBFDF91CF910895CF93DF9326
:10139000CDB7DEB726970FB6F894DEBF0FBECDBF30
:1013A0009E838D831C821B821DC08D818A838D81CB
:1013B0009E81892F99278983698185E00E94EF00AA
:1013C0006A8186E00E94EF0060E087E00E94EF0003
:1013D0008D819E814E969E838D838B819C8101960B
:1013E0009C838B838B819C8188309105F0F22696BB
:1013F0000FB6F894DEBF0FBECDBFDF91CF91089539
:10140000CF93DF93CDB7DEB727970FB6F894DEBF43
:101410000FBECDBF9E838D836F831C821B8223C032
:101420008D818A838D819E81892F99278983698106
:1014300085E00E94EF006A8186E00E94EF008F81C4
:101440009927FC01E35DFE4F8081682F87E00E94B1
:10145000EF008D819E814E969E838D838B819C8132
:1014600001969C838B838B819C8188309105C0F28F
:1014700027960FB6F894DEBF0FBECDBFDF91CF9198
:101480000895CF93DF93CDB7DEB726970FB6F894C4
:10149000DEBF0FBECDBF809150049091510426E174
:1014A00030E0B9010E943712CB019E838D838D817C
:1014B0009E8199230CF452C08D819E812AE030E0F8
:1014C000B9010E943712CB018A838D819E812AE067
:1014D00030E0B9010E94371289838981869589831A
:1014E0008A81282F332787E090E0AC01421B530B01
:1014F0009A018EE190E0AC01249FC001259F900DE0
:10150000349F900D11240A969C838B8320910B01AC
:1015100030910C018B819C818217930761F080913F
:101520000B0190910C010E94110B8B819C816981B0
:101530000E94740B0AC09091B0038981981729F01A
:101540008B819C8169810E94740B89818093B00397
:101550008B819C8190930C0180930B018D819E81E6
:1015600099230CF055C08D819E81909581959F4F58
:101570009E838D838D819E812AE030E0B9010E9497
:101580003712CB018A838D819E812AE030E0B90138
:101590000E9437128983898186958C5F89838A812D
:1015A000282F33278EE190E0AC01249FC001259FB6
:1015B000900D349F900D112486509F4F9C838B83F8
:1015C00020910B0130910C018B819C818217930734
:1015D00061F080910B0190910C010E94110B8B81A5
:1015E0009C8169810E94740B0AC09091B00389812B
:1015F000981729F08B819C8169810E94740B8981E5
:101600008093B0038B819C8190930C0180930B019C
:1016100026960FB6F894DEBF0FBECDBFDF91CF91F7
:101620000895CF93DF93CDB7DEB726970FB6F89422
:10163000DEBF0FBECDBF9E838D838D819E819C8337
:101640008B8318C08B818A838B819C81892F9927FA
:101650008983698185E00E94EF006A8186E00E94AB
:10166000EF0060E087E00E94EF008B819C81019693
:101670009C838B838D819E819C01275F3F4F8B8153
:101680009C8182179307F0F28091B003282F3327B3
:10169000C901880F991F820F931FFC01EF5EFE4F57
:1016A00080818823C1F08D819E8182969C838B836B
:1016B0008B818A838B819C81892F9927898369817A
:1016C00085E00E94EF006A8186E00E94EF0060E002
:1016D00087E00E94EF0026960FB6F894DEBF0FBE9B
:1016E000CDBFDF91CF910895CF93DF93CDB7DEB714
:1016F00027970FB6F894DEBF0FBECDBF9E838D83B4
:101700006F838D819E819C838B8324C08B81898391
:101710008B819C81892F99278A836A8185E00E9429
:10172000EF00698186E00E94EF008F81282F332728
:10173000C901880F991F820F931FFC01E15FFE4FC3
:101740008081682F87E00E94EF008B819C81019649
:101750009C838B838D819E819C01275F3F4F8B8172
:101760009C818217930790F28D819E8104969C83C1
:101770008B838B8189838B819C81892F99278A8395
:101780006A8185E00E94EF00698186E00E94EF0097
:101790008F81282F3327C901880F991F820F931F2C
:1017A000FC01E05FFE4F8081682F87E00E94EF0020
:1017B0008F81282F3327C901880F991F820F931F0C
:1017C000FC01EF5EFE4F8081882321F18D819E8197
:1017D00082969C838B838B8189838B819C81892FCB
:1017E00099278A836A8185E00E94EF00698186E0FB
:1017F0000E94EF008F81282F3327C901880F991F7E
:10180000820F931FFC01EF5EFE4F8081682F87E0FF
:101810000E94EF0027960FB6F894DEBF0FBECDBF33
:10182000DF91CF910895CF93DF93CDB7DEB760E01E
:1018300085E00E94EF0063E886E00E94EF0060E927
:1018400087E00E94EF0060E085E00E94EF0064E81E
:1018500086E00E94EF0061E987E00E94EF0060E00F
:1018600085E00E94EF0065E886E00E94EF0062E9F3
:1018700087E00E94EF0060E085E00E94EF0066E8EC
:1018800086E00E94EF0063E987E00E94EF0060E0DD
:1018900085E00E94EF0067E886E00E94EF0064E9BF
:1018A00087E00E94EF0060E085E00E94EF0068E8BA
:1018B00086E00E94EF0065E987E00E94EF0060E0AB
:1018C00085E00E94EF0069E886E00E94EF0066E98B
:1018D00087E00E94EF0060E085E00E94EF006AE888
:1018E00086E00E94EF0067E987E00E94EF0060E079
:1018F00085E00E94EF0061EA86E00E94EF0068E95F
:1019000087E00E94EF0060E085E00E94EF0062EA5D
:1019100086E00E94EF0069E987E00E94EF0060E046
:1019200085E00E94EF0063EA86E00E94EF006AE92A
:1019300087E00E94EF0060E085E00E94EF0064EA2B
:1019400086E00E94EF006BE987E00E94EF0060E014
:1019500085E00E94EF0065EA86E00E94EF006CE9F6
:1019600087E00E94EF0060E085E00E94EF0066EAF9
:1019700086E00E94EF006DE987E00E94EF0060E0E2
:1019800085E00E94EF0067EA86E00E94EF006EE9C2
:1019900087E00E94EF0060E085E00E94EF0068EAC7
:1019A00086E00E94EF006FE987E00E94EF0060E0B0
:1019B00085E00E94EF006FEB86E00E94EF0060EA96
:1019C00087E00E94EF0060E085E00E94EF0060EC9D
:1019D00086E00E94EF0061EA87E00E94EF0060E08D
:1019E00085E00E94EF0061EC86E00E94EF0062EA71
:1019F00087E00E94EF0060E085E00E94EF0062EC6B
:101A000086E00E94EF0063EA87E00E94EF0060E05A
:101A100085E00E94EF0063EC86E00E94EF0064EA3C
:101A200087E00E94EF0060E085E00E94EF0064EC38
:101A300086E00E94EF0065EA87E00E94EF0060E028
:101A400085E00E94EF0065EC86E00E94EF0066EA08
:101A500087E00E94EF0060E085E00E94EF0066EC06
:101A600086E00E94EF0067EA87E00E94EF0060E0F6
:101A700085E00E94EF006DED86E00E94EF0068EACD
:101A800087E00E94EF0060E085E00E94EF006EEDCD
:101A900086E00E94EF0069EA87E00E94EF0060E0C4
:101AA00085E00E94EF006FED86E00E94EF006AEA99
:101AB00087E00E94EF0060E085E00E94EF0060EEAA
:101AC00086E00E94EF006BEA87E00E94EF0060E092
:101AD00085E00E94EF0061EE86E00E94EF006CEA74
:101AE00087E00E94EF0060E085E00E94EF0062EE78
:101AF00086E00E94EF006DEA87E00E94EF0060E060
:101B000085E00E94EF0063EE86E00E94EF006EEA3F
:101B100087E00E94EF0060E085E00E94EF0064EE45
:101B200086E00E94EF006FEA87E00E94EF0060E02D
:101B300085E00E94EF006BEF86E00E94EF0060EB13
:101B400087E00E94EF0060E085E00E94EF006CEF0C
:101B500086E00E94EF0061EB87E00E94EF0060E00A
:101B600085E00E94EF006DEF86E00E94EF0062EBDF
:101B700087E00E94EF0060E085E00E94EF006EEFDA
:101B800086E00E94EF0063EB87E00E94EF0060E0D8
:101B900085E00E94EF006FEF86E00E94EF0064EBAB
:101BA00087E00E94EF0061E085E00E94EF0060E0C6
:101BB00086E00E94EF0065EB87E00E94EF0061E0A5
:101BC00085E00E94EF0061E086E00E94EF0066EB96
:101BD00087E00E94EF00DF91CF910895CF93DF93CC
:101BE000CDB7DEB764970FB6F894DEBF0FBECDBF9A
:101BF00083E090E09C8B8B8B1A82198283E990E0C2
:101C00009C838B831092B303CFC08B899C89FC018A
:101C1000EC54FC4F80819927CD979A8B898B8B89C7
:101C20009C8901969C8B8B8B8B899C89FC01EC5445
:101C3000FC4F80819927CD97988B8F878B899C89C2
:101C400001969C8B8B8B8B899C89FC01EC54FC4FFF
:101C500080819927CD979E878D878B899C89019656
:101C60009C8B8B8B8B899C89FC01EC54FC4F808175
:101C70009927CD979C878B878B899C8901969C8B14
:101C80008B8B89899A899C01220F331F220F331F66
:101C90008F8598899595879595958795959587953D
:101CA00095958795822B932B9A8789878F8598891D
:101CB0008F7090709C0122953295307F3227207F63
:101CC00032278D859E859595879595958795822B4D
:101CD000932B98878F838D859E85837090709C0150
:101CE0000024369527950794369527950794322F2B
:101CF000202D8B859C85822B932B9E838D838B81BE
:101D00009C8101979C838B838B819C812FEF8F3FDC
:101D1000920709F44EC089819A819C0180919F03AA
:101D20009091A003F901E80FF91F898580838981CB
:101D30009A8101969A8389838B819C8101979C83E8
:101D40008B838B819C812FEF8F3F920791F189814B
:101D50009A819C0180919F039091A003F901E80F63
:101D6000F91F8F81808389819A8101969A83898363
:101D70008B819C8101979C838B838B819C812FEF2E
:101D80008F3F9207B1F089819A819C0180919F03D6
:101D90009091A003F901E80FF91F8D81808389815B
:101DA0009A8101969A8389838B819C81009709F09F
:101DB0002CCF64960FB6F894DEBF0FBECDBFDF9177
:101DC000CF910895CF93DF93CDB7DEB7E9E2F0E08E
:101DD00082E28083E0E4F0E01082E0E2F0E082E280
:101DE0008083ECE5F0E01082A2E3B0E0E2E3F0E013
:101DF000808181608C93A8E3B0E0E8E3F0E080812B
:101E000084608C93EAE2F0E088E98083E0E4F0E02B
:101E100086E88083EBE2F0E082EC8083E1E2F0E0B0
:101E200088E98083ECE5F0E086E88083E2E2F0E098
:101E300082EC8083DF91CF910895CF93DF93CDB76C
:101E4000DEB721970FB6F894DEBF0FBECDBF8983F2
:101E5000EBE2F0E080819927807290700097C1F3E7
:101E6000ECE2F0E08981808321960FB6F894DEBF22
:101E70000FBECDBFDF91CF910895CF93DF93CDB744
:101E8000DEB726970FB6F894DEBF0FBECDBF9E8398
:101E90008D838D819E81DC01FD0101900020E9F799
:101EA0003197CF018A1B9B0B9C838B831A821982EB
:101EB0000FC029813A818D819E81F901E80FF91FB8
:101EC00080810E941D0F89819A8101969A8389835E
:101ED00029813A818B819C818217930750F78091E9
:101EE000A1030E941D0F8091A2030E941D0F269640
:101EF0000FB6F894DEBF0FBECDBFDF91CF9108952E
:101F0000CF93DF93CDB7DEB766970FB6F894DEBFF9
:101F10000FBECDBF9E8B8D8B8D899E894AE050E090
:101F20009E012F5F3F4FB9010E940612CE0101961C
:101F30000E943D0F66960FB6F894DEBF0FBECDBF70
:101F4000DF91CF910895CF93DF93CDB7DEB722977E
:101F50000FB6F894DEBF0FBECDBF8A8387E08983BA
:101F60001FC08A81482F55278981282F332727FDB5
:101F7000309581E090E0022E02C0880F991F0A94EC
:101F8000E2F7842395231816190624F481E30E94AE
:101F90001D0F03C080E30E941D0F8981815089833A
:101FA00089818823F4F68091A1030E941D0F8091FE
:101FB000A2030E941D0F22960FB6F894DEBF0FBE3B
:101FC000CDBFDF91CF9108951F920F920FB60F9260
:101FD00011242F933F938F939F93AF93BF93EF93CE
:101FE000FF93CF93DF93CDB7DEB72297DEBFCDBF90
:101FF000E3E2F0E0808180939004809190048D3042
:10200000D1F48091B2038130B1F4A5E3B0E0E5E30F
:10201000F0E08081877F8C931092B20381E08093FF
:10202000B30380914A04992720919004FC01EC5459
:10203000FC4F208348C08091B203282F33273A8376
:10204000298389819A81009731F029813A81213051
:10205000310521F138C080919004833271F4809170
:10206000B303882351F481E08093B203A5E3B0E089
:10207000E5E3F0E0808188608C9310924A0430910F
:102080004A04832F992720919004FC01EC54FC4FC3
:102090002083832F8F5F80934A0415C080914A0468
:1020A000992720919004FC01EC54FC4F20838091EF
:1020B0004A04863930F480914A048F5F80934A0441
:1020C00002C01092B2032296F894DEBFCDBFDF911A
:1020D000CF91FF91EF91BF91AF919F918F913F91E0
:1020E0002F910F900FBE0F901F901895CF93DF93F5
:1020F000CDB7DEB76E970FB6F894DEBF0FBECDBF7B
:102100002091500430915104CE010B964AE050E0EA
:10211000BC01C9010E94061280E4898384E48A8399
:1021200080E38B831C82CE010B96DC01FD010190C4
:102130000020E9F73197CF018A1B9B0B9E01255F99
:102140003F4FAC01B901CE0101960E94F611CE01BC
:102150000196DC01FD0101900020E9F731979F0114
:102160002A1B3B0BCE010196820F931FFC0183E2D9
:1021700090E091838083CE0101960E943D0F2091D3
:10218000520430915304CE010B964AE050E0BC015A
:10219000C9010E94061280E4898384E48A8381E372
:1021A0008B831C82CE010B96DC01FD010190002087
:1021B000E9F73197CF018A1B9B0B9E01255F3F4FAB
:1021C000AC01B901CE0101960E94F611CE01019633
:1021D000DC01FD0101900020E9F731979F012A1BE6
:1021E0003B0BCE010196820F931FFC0183E290E02E
:1021F00091838083CE0101960E943D0F20915A0465
:1022000030915B04CE010B964AE050E0BC01C9015D
:102210000E94061280E4898388E68A838DE38B839B
:102220001C82CE010B96DC01FD0101900020E9F734
:102230003197CF018A1B9B0B9E01255F3F4FAC015D
:10224000B901CE0101960E94F611CE010196DC0182
:10225000FD0101900020E9F731979F012A1B3B0BFC
:10226000CE010196820F931FFC0183E290E09183DF
:102270008083CE0101960E943D0F2091620430912F
:102280006304CE010B964AE050E0BC01C9010E94F4
:10229000061280E4898386E58A838CE68B831C8220
:1022A000CE010B96DC01FD0101900020E9F731978A
:1022B000CF018A1B9B0B9E01255F3F4FAC01B901EB
:1022C000CE0101960E94F611CE010196DC01FD01BE
:1022D00001900020E9F731979F012A1B3B0BCE01AB
:1022E0000196820F931FFC0183E290E0918380832B
:1022F000CE0101960E943D0F2091AC033091AD03B9
:10230000CE010B964AE050E0BC01C9010E940612C2
:1023100080E4898386E58A8381E48B831C82CE01F5
:102320000B96DC01FD0101900020E9F73197CF0108
:102330008A1B9B0B9E01255F3F4FAC01B901CE016B
:1023400001960E94F611CE010196DC01FD0101907B
:102350000020E9F731979F012A1B3B0BCE01019624
:10236000820F931FFC0183E290E091838083CE0172
:1023700001960E943D0F6E960FB6F894DEBF0FBE19
:10238000CDBFDF91CF910895CF93DF93CDB7DEB767
:10239000A5E3B0E0E5E3F0E0908182E089278C934B
:1023A000DF91CF910895CF93DF93CDB7DEB78091C2
:1023B000AB038130C1F48091AA03813051F4A5E3CD
:1023C000B0E0E5E3F0E080818E7F8C931092AA0369
:1023D0000AC0A5E3B0E0E5E3F0E0808181608C9382
:1023E00081E08093AA03DF91CF910895FB01DC0186
:1023F0000D900020E9F711974150504028F00190CE
:1024000000200D92C9F708951C920895FB019F01C9
:10241000E8944230C4F04532B4F44A3029F497FBD2
:102420001EF4909581959F4F642F77270E944A1242
:10243000805D8A330CF0895D8193CB010097A1F711
:1024400016F45DE251931082C9010C942712DC014D
:10245000FC0101900020E9F73297AE17BF0730F476
:102460007C916081708331976D93F7CF089597FBCE
:10247000092E07260AD077FD04D00CD006D0002004
:102480001AF4709561957F4F0895F6F790958195B0
:102490009F4F0895AA1BBB1B51E107C0AA1FBB1F7A
:1024A000A617B70710F0A61BB70B881F991F5A95E0
:0C24B000A9F780959095BC01CD0108951E
:1024BC0001125A2C294400000A3100230023005435
:1024CC006466536365526200516100506000506055
:1024DC000051610052620053636554646667686919
:1024EC006A6B6B6A696867AAAAAAAAAAAAAAAAAA04
:1024FC00AAAAAAAAAAAAAAAAA9AAAAA9AAAAA5AA37
:10250C00AAA5AAAA95AAAA95AAAA55AAAA55AAA9F9
:10251C0056AAA556AA955AAA556AA955AA555595CB
:10252C006A55956A5555AA5555A95555A95556A993
:10253C005556A55556A5555A95555A95556A9555BE
:10254C006A5555AA5555A95555A55555A555559591
:10255C00555555555555555555555555555555551F
:10256C00555555555555555555555555555555550F
:10257C0055555555555555555555555555555555FF
:10258C00555555555555555555555555555555AA9A
:10259C00555A6A95565AA55556A95555AA55556A70
:1025AC00A5555AA95556AA5555AA55555A55555675
:1025BC0055555555555555555555555555555555BF
:1025CC0055555555555555AA9565AA5955AA65960B
:1025DC006AAA5656AA5A55AAAA555AAA5555AAA530
:1025EC00555AAA5555AA95556AAA555AAAA555AA37
:1025FC00AA5556AA55556A5555555555555555A56F
:10260C00AAAAA5A5AAA596AAA55AAA965AAA965A5E
:10261C0095965AAAAA5AAAAAAAAA6AAAAA556AAAAC
:10262C00555555555555955555AAA955AAAAAA6A51
:10263C00AAAA556AAA5555AAAA5AA59696A5A696C7
:10264C00A59AA5A59AA5A5AAA5A9A5A9A955AAAA79
:10265C00AAAAAAAAA9AAA9555555555555555555CD
:10266C0056556AAAAAAAAAAAAAAAAAA95555555AF7
:10267C0096AA5A95AA6AA5AAAAAAA9AAAAA56AAAB2
:10268C0055AAA555AA5555A5555A55556A5556AA34
:10269C00556AA95AAAA5AAAA55AA9555A955555538
:1026AC0055555555555555A555AA9556A9555AA53F
:1026BC00556A9555AA555AA9556AA555AA9555AA6C
:1026CC005555A5555595555555555555555555551E
:1026DC00555555555555555555555555555555559E
:1026EC00555555555555555555555555555555558E
:1026FC00555555555555555555555555555555557E
:10270C00555555555555555555555555555555556D
:10271C005555555555555555555955559655556508
:10272C0056555556565566A9555A555556555556DE
:10273C0056A95959565955595955555955555965BB
:10274C0055596555655A566555A955555555554EA6
:04275C00040D0A005E
:00000001FF
